:020000040000FA
:1000000032EF03F0F76A140FF66E000EF7220900C4
:10001000F55012003031372055534220696E746517
:100020007266616365204654323435424D200A0DB4
:100030000000EA6A1B0EE96EEF500FE0010E016E40
:10004000006A002EFED7012EFBD74A0E006E002E4E
:10005000FED700000000EF2EF1D7000C086A076AF7
:10006000060E946E829A116A115226E1100E1A6ED3
:100070001A521EE08290020E1B6EDBDF828082A489
:1000800012D0010E1A5C1B6E036A010E026E1B5029
:10009000006E05E0D89002360336002EFBD70250E2
:1000A000071203500812020E1B6EC3DF1A06E0D7B8
:1000B000116A07B4112AD8D7020E946E195202E1C0
:1000C000829403D01952D8A48284100E1A6E1A5248
:1000D0000AE08290020E1B6EACDF8280020E1B6E65
:1000E000A8DF1A06F4D78290828A060E946E4BEF30
:1000F00002F08E0E006E1AC001F019C002F0036A01
:100100001AAE05D0011E021E022A01E1012A015287
:1001100009E102C001F0026A080E005E015202E12C
:10012000006A0AD0D89001BE04D00236013600061B
:10013000F9D71ABE01D0019E000080EF02F01D50D9
:1001400069E0006E215066E0002604E3810E00267F
:1001500061E204D07F0E005E5DE35CE01EC025F02E
:100160002250251A1E8E228E20502402F4CF27F012
:100170001F502302F4CF03F0F3CF26F02402F350F4
:100180002726F4502622000E032220502302F3508B
:100190002726F4502622000E026A032202221E5055
:1001A0002402F3502626F4500322000E02221E5091
:1001B0002302F3500326F4500222000E01222050A5
:1001C0002202F3502626F4500322016A000E022276
:1001D00001221F502202F3500326F4500222000E87
:1001E00001221E502202F3500226F4500122002A5E
:1001F00001BE05D026360336023601360006000E53
:1002000026AE03D0032A0222012225BE018E25AE8E
:10021000019E04D0006A016A026A036A000096EF38
:1002200002F0800ED8B2261A2B6A2C6A22C02AF05D
:1002300026502A1A2150D8B4DED0296E29C000F0E9
:100240002550D8B4E1D0295ED8B482D001E23DD0A7
:1002500026C02FF02F8E27C02EF028C02DF02C6A3C
:10026000D8902F322E322D322C32292EF8D72AAEAA
:1002700003D02B80DDD02B9029902B88EA6A240EA6
:10028000E96EE9D02B982ABE0AD029A013D02F32CC
:100290002E322D322C32002AD8B4C5D00BD02FBE2E
:1002A0000CD0D8902C362D362E362F360006D8B4EA
:1002B000BAD0F5D72B8C6BD02B9C22C02AF022AE63
:1002C00002D02F8EA9D02F9EA7D025C029F025C0FF
:1002D00000F02150295E22C02FF02F8E23C02EF077
:1002E00024C02DF02C6AD8902F322E322D322C3291
:1002F000292EF8D72AAE03D02B829AD02B922990A0
:100300002B8AEA6A280EE96EA6D02B9A2ABE0AD05A
:1003100029A013D02F322E322D322C32002AD8B4FD
:1003200082D00BD02FBE0CD0D8902C362D362E3646
:100330002F360006D8B477D0F5D72B8E28D02B9E39
:1003400026C02AF026AE02D02F8E66D02F9E64D013
:1003500026C02FF02F8E27C02EF028C02DF02AAEF9
:1003600004D02F9E2B8464D02B942C6A2990EA6AA7
:10037000240EE96E70D02ABE1CD022C02AF029A01B
:1003800006D02F322E322D322C32002A4CE02CAEE9
:100390000BD02D2A09E12E2A07E12F2A05E12F3261
:1003A0002E322D32002A3FE02BBC86D72BBEC7D77A
:1003B0001CD0800E2F1A2FAE04D03AD026C02AF0BF
:1003C0000AD022C02AF02F5206E12E5204E12D520B
:1003D00002E1006A21D02FBE08D0D8902C362D36ED
:1003E0002E362F36002EF7D71ED02AAE02D02F8EF3
:1003F00013D02F9E11D025C000F026C02FF027C0AB
:100400002EF028C02DF008D021C000F022C02FF01F
:1004100023C02EF024C02DF02FC001F02EC002F01A
:100420002DC003F034D0006A016A026A036A2FD03B
:100430002C6A2D1E2E1E2F1E2C1E2C2A05E12D2A65
:1004400003E12E2A01E12F2A2BB015D72BB256D764
:100450002BB48AD7B3D7EF502D2605E32E2A03E11C
:100460002F2AD8B42980ED52EF502E2603E32F2AED
:10047000D8B42980ED52EF50EFBE01D0800A2F266C
:10048000D8B029802BB8FED62BBA3FD774D700003E
:10049000000C196AE3D5060E946E116A115229E117
:1004A000829A066A056A100E186E185218E0829039
:1004B000828082A412D0010E185C196E036A010EAC
:1004C000026E1950006E05E0D89002360336002EF9
:1004D000FBD702500512035006121806E6D7828A8F
:1004E000000E05B4010E010803E1010E116E01D0EA
:1004F000D5D7F80E051606C01AF005C019F0F9D5C3
:1005000000C019F001C01AF002C01BF003C01CF0BB
:1005100003C020F002C01FF001C01EF000C01DF09B
:10052000246A236A226A780E216E09D600C01DF063
:1005300001C01EF002C01FF003C020F0D88203C02B
:1005400024F002C023F001C022F000C021F0660EAA
:10055000286E276E060E266E800E256E62DE03C0A4
:100560000CF002C00BF001C00AF000C009F0D88204
:100570000CC024F00BC023F00AC022F009C021F007
:10058000660E286E276E260E266E7F0E256E49DEBD
:1005900003C00CF002C00BF001C00AF000C009F06B
:1005A0006BEF03F081BA04D01EC083FF818881986D
:1005B000000C81BA55D0000E956E136A13500108D5
:1005C0001EE3036A1350140F016E000E032201C0D4
:1005D0001CF003C01DF0050E1324016E036AD8B091
:1005E000032A01C0E9FF03C0EAFFEFCF1EF01DC0E0
:1005F000EAFF1CC0E9FF1EC0EFFF132ADFD7040E7D
:10060000136E135212E0010E135C180F016E036A91
:10061000D8B0032A01C0E9FF03C0EAFFEFCF1CF006
:100620001CC01EF0BFDF1306ECD7020E136E135270
:1006300004E01E6AB7DF1306FAD7020E136E1352D8
:100640000FE0010E135C036A140FE96E000E032025
:10065000EA6EEFCF1DF01DC01EF0A4DF1306EFD72A
:1006600075EF03F0F86AD09EFE0E006E060E016E66
:10067000EA6A020EE96EEF6AE92AD8B4EA2A002E85
:10068000FAD7012EF8D7EA6AE96AC180C182C1842B
:10069000C1960C0EAF6E260EAC6E900EAB6E000EB9
:1006A000926E600E936E020E946EFF0E956E969093
:1006B00096929694186A1850A5DC182A006E00507D
:1006C0009EA8FED7AD6E1C0E185CF5E18186819860
:1006D000126A818EDED6819E760E1B6E540E1A6EC5
:0E06E000320E196E100E186E64D7F3D7030099
:020000040030CA
:0E00000000210C0E000180000FC00FE00F4029
:00000001FF
